:100000000C9450010C9479010C9479010C947901B1
:100010000C9479010C9479010C9479010C94CE0222
:100020000C9479010C9479010C9479010C94790168
:100030000C9479010C9479010C9479010C94790158
:100040000C9479010C9479010C947C030C94790143
:100050000C9439030C9479010C9479010C94790176
:100060000C9479010C947901437934436F6465A051
:10007000032011B0011020F0FF000100025F020018
:10008000FFFF003D0002290240FFFF0001000114B4
:1000900002F0FFFF00070000E901F8FFFF00010088
:1000A00001D601FAFFFF00010001C301FCFFFF00C0
:1000B0000200017B0120650501806D060101140627
:1000C000010000000002000002000000010000002A
:1000D0000100000001020F06030000000200000002
:1000E0000200000002206505014065050104670665
:1000F000040000000310380603080F06000000008B
:100100000400000004005EBCE2613FDD83C29C7E0F
:1001100020A3FD1F419DC3217FFCA2401E5F01E380
:10012000BD3E6082DC237D9FC1421CFEA0E1BF5D1D
:100130000380DE3C62BEE0025CDF81633D7C22C066
:100140009E1D43A1FF4618FAA427799BC584DA387F
:1001500066E5BB5907DB856739BAE406581947A538
:10016000FB7826C49A653BD987045AB8E6A7F91BE1
:1001700045C6987A24F8A6441A99C7257B3A64861E
:10018000D85B05E7B98CD2306EEDB3510F4E10F24B
:10019000AC2F7193CD114FADF3702ECC92D38D6FE8
:1001A00031B2EC0E50AFF1134DCE90722C6D33D1B5
:1001B0008F0C52B0EE326C8ED0530DEFB1F0AE4CCE
:1001C0001291CF2D73CA947628ABF517490856B40F
:1001D000EA6937D58B5709EBB536688AD495CB29B0
:1001E00077F4AA4816E9B7550B88D6346A2B759769
:1001F000C94A14F6A8742AC896154BA9F7B6E80A96
:1002000054D7896B35020403050606070708080959
:1002100009015C0601000000000000000000000071
:1002200000200000000200000200000001000000A9
:1002300001020000030000000200000002000000B4
:10024000024000000020000000800000000458066A
:100250000410340603080000000000000400000041
:1002600004015B437934696E6F20556E6F204261E3
:100270007369635D000000000000000000000000E2
:10028000000000000000000000000000000000006E
:10029000000000000000000000000000000000005E
:1002A00011241FBECFEFD8E0DEBFCDBF14BE0FB606
:1002B000F894A89580916000886180936000109206
:1002C00060000FBE11E0A0E0B1E0E2E9F9E102C098
:1002D00005900D92A830B107D9F723E0A8E0B1E06E
:1002E00001C01D92AE35B207E1F70E94F70A0C94E7
:1002F000C70C0C940000EF92FF920F931F93CF93C3
:10030000DF9300D000D0CDB7DEB77C018B010E9417
:10031000800A9A838983CE0101960E9410058B83FF
:10032000CE0101960E9413058C83AE014D5F5F4F95
:10033000B801C7010E94CB0A8B8189838C818A8393
:10034000CE0101960E942405882321F0C8010E9455
:1003500031050EC0CE0101960E9416058823B1F327
:1003600089819A810E947E0ACE0101960E94660BC5
:100370000F900F900F900F90DF91CF911F910F91E1
:10038000FF90EF900895CF93DF93EB01CB010E9494
:100390004305FC0180818E3521F4DF91CF910C94CF
:1003A000C303CE01DF91CF910C943105CF93DF933E
:1003B000EB01CB010E944305FC0180818E3521F4C5
:1003C000DF91CF910C94C003CE01DF91CF910C94BB
:1003D0003105FF920F931F93CF93DF93EC018B01B5
:1003E000CB010E943A05F62ECE010E94C50AF61AEC
:1003F000D0E0CD2FCF0DC8010E944005D81770F472
:10040000C8010E944505EC2FF0E0E159FF4FE4914F
:10041000DC01AD0FB11DEC93DF5FEBCFDF91CF912E
:100420001F910F91FF900895CF93DF93EB01CB01C4
:100430000E944305FC0180818E3531F40E941D0B22
:10044000DF91CF910C94C003CE01DF91CF910C943A
:100450003105EF92FF920F931F93CF93DF93CDB7A8
:10046000DEB7ED970FB6F894DEBF0FBECDBF8C019F
:100470007B014DE350E0BE016F5F7F4F8BE090E06A
:100480000E94140BAE014F5F5F4FB701C8010E947D
:10049000CB0A1DAE4DE350E06BE070E0CE0101965B
:1004A0000E94160BED960FB6F894DEBF0FBECDBFBF
:1004B000DF91CF911F910F91FF90EF9008950F93CF
:1004C0001F93CF93DF931F92CDB7DEB78B01CB0184
:1004D0000E943705811110C041E050E0BE016F5FFE
:1004E0007F4F8AE090E00E94140BC8010E944505EE
:1004F0002981FC01208315C0C8010E944305FC012D
:1005000091E08081811101C090E0998341E050E049
:100510006AE070E0CE0101960E94160B89810E946C
:100520008B040F90DF91CF911F910F910895CF937E
:10053000DF931F92CDB7DEB786E790E00E94620A94
:100540000E94410B0E947E0A41E050E0BE016F5FB5
:100550007F4F8AE090E00E94140B89810E948B04F7
:100560000F90DF91CF91089508950895F89498E041
:1005700088E10FB6F894A895809360000FBE909321
:100580006000E0E0F1E080E099E08193E030F9077D
:10059000E0F3FFCF87FF01C0789408951F920F9278
:1005A0000FB60F9211242F938F939F93EF93FF9386
:1005B00080910B01843021F410920B018BE204C076
:1005C0008F5F80930B018AE28093B30080912902B0
:1005D00090912A02019690932A0280932902809199
:1005E000090190910A010196883E23E0920729F0C3
:1005F00090930A01809309010DC010920A01109294
:100600000901809127029091280201969093280277
:10061000809327028091D80186958695869590E0F3
:100620000497ECF48091D801887F98E0980F80912E
:10063000D8018770892B8093D8018091D801869545
:100640008695869590E0049754F0E0910E01F0E0D5
:10065000EE0FFF1FE05FFE4F808181608083FF917E
:10066000EF919F918F912F910F900FBE0F901F9040
:1006700018951F920F920FB60F9211248F939F938C
:10068000EF93FF938091D80181FD07C08091D8013D
:1006900084608093D8011092DA018091D8018D7F17
:1006A0008093D8018091DB019091DA01911106C00D
:1006B0009091D8019E7F9093D80113C0E82FF0E06D
:1006C000E452FE4F90819093D90190819093C6009F
:1006D0008F5F8B3409F480E09091DA019150909310
:1006E000DA018093DB01FF91EF919F918F910F9041
:1006F0000FBE0F901F9018951F920F920FB60F927A
:1007000011248F939F93EF93FF939091C600809154
:10071000D80187708093D8018091D80180FF09C0EB
:100720008091D901981305C08091D801826080938F
:10073000D80180910E01E82FF0E0EE0FFF1FE05F7F
:10074000FE4F91838F5F843609F480E090910F0112
:1007500089130BC0E0910E01F0E0EE0FFF1FE05F88
:10076000FE4F80818160808302C080930E01FF91E3
:10077000EF919F918F910F900FBE0F901F90189542
:1007800010920D01089581E080930D010895CF939B
:10079000DF938FB7F894C0912902D0912A020E946A
:1007A000CA02CE01DF91CF9108959C01CB01B9011E
:1007B0000C94950C0C94A50CCF938FB7F894909152
:1007C000D80190FD0AC02091D8012695269526953E
:1007D00030E0C1E0243031050CF4C0E00E94CA02D0
:1007E0008C2F8170CF910895CF93DF93C82F8FB74F
:1007F000F894D091DA010E94CA02DB34C1F38FB7BA
:10080000F8949091D80192FD24C09091D80190FF66
:1008100012C0E091DB019091DA01E90FEB3408F0AE
:10082000EB54F0E0E452FE4FC0839091DA019F5FF9
:100830009093DA010EC09091D80191609093D80105
:100840009091D8019D7F9093D801C093D901C09316
:10085000C600DF91CF910C94CA02CF938FB7F89462
:10086000C091D801C1700E94CA028C2FCF91089507
:10087000CF938FB7F894C091D801C2FBCC27C0F9B1
:100880009091D8019B7F9093D8010E94CA028C2F2F
:10089000CF910895CF93DC018FB7F894C0E0909189
:1008A0000F01E92FF0E0EE0FFF1FE05FFE4F208108
:1008B00020FD0EC020910E01921751F0319620813B
:1008C0002C939F5F943609F490E090930F01C1E060
:1008D0000E94CA028C2FCF910895CF938FB7F894BE
:1008E00090910F01E92FF0E0EE0FFF1FE05FFE4F48
:1008F000C081C17020910E01921719F090819E7FE6
:1009000090830E94CA0281E08C27CF91089589E1EB
:1009100080930C01089580930001811101C05F98BC
:10092000089580910D0181110E94B602F8949FE014
:1009300088E10FB6F894A895809360000FBE90935D
:10094000600081E084B915B817B818B880E88AB992
:100950001BB88DED90E001970000E9F783E290E08D
:100960009093C5008093C4001092C00088ED8093DE
:10097000C10096E09093C20082E08093B000909313
:10098000B1009AE29093B3008093700078948093C2
:100990000D01089581E090910D01923009F080E001
:1009A00008950E94C7032091080130E0AC0155274B
:1009B00024173507D9F080930801A89520910001EC
:1009C000222341F0807892708038910511F45F9A6B
:1009D00001C05F9880910C01882341F08150809381
:1009E0000C01882311F0289A0895289808950E94F0
:1009F0002D048111FCCF80910D01882361F081309D
:100A000061F4E0E0F8E7859194918C30944929F401
:100A10000C94023C08950E94B6020895962F089502
:100A2000FC0180810895FC0181810895FC01808191
:100A30008F3F39F491E081818F3F09F490E0892F55
:100A400001C081E081700895FC018081882331F02C
:100A500091E08181811190E0892F01C081E0817056
:100A60000895FC0110820895FC0180810895FC0125
:100A700081810895FC016481758186819781089543
:100A8000FC01808508950996089509960895DC0172
:100A90009BE4E0EDF2E001900D929A95E1F710925F
:100AA000CF020895EEE2F2E0818180958370806C40
:100AB00081838281848383818583A3E0B1E08C91EB
:100AC000828311968C91838308950E94520510921F
:100AD0002E020895EF92FF920F931F93CF93DF930F
:100AE000DC012C9130E08901E4E0000F111FEA9550
:100AF000E1F7A0E0B0E0C0E0D0E0F801EA0FFB1FB2
:100B0000E40FF51FF490FF2061F1FB01E080EF2D71
:100B1000EE2111F1220F331F220F331F2C0F3D1F27
:100B2000220F331F220F331FF9013196E40FF51FF7
:100B300065917491F9013396E40FF51FE491DC019E
:100B4000EC936115710569F0FB01DF91CF911F9165
:100B50000F91FF90EF90099421961496A031B10562
:100B600061F6DF91CF911F910F91FF90EF90089563
:100B7000FC01DB0181E090819A3A09F080E08C93DE
:100B80008181815C91E0823008F490E011969C9321
:100B90001197848112968C931297858113968C936A
:100BA0001397468150E060E070E0BA015527442772
:100BB0008085480F511D611D711D878190E0982F20
:100BC0008827480F591F611D711D14964D935D9321
:100BD0006D937C931797918518969C9318978181B4
:100BE00080FF09C03A96199680E0891721F021917B
:100BF0002D938F5FFACF08951F93CF93DF93EC016E
:100C0000162F0E94C703810F911D009711F481E0F8
:100C100090E099838883DF91CF911F9108956AEFC7
:100C20008BE792E00C94FC058EE292E00E9447056F
:100C300062E389E792E00C94FC05CF93DF93EC012B
:100C40000E94C70383709927019690910101890F33
:100C5000803108F083E08093010160910101CE01B1
:100C6000DF91CF910C94FC0589EC92E00C941D0669
:100C700089E792E00C941D060F931F93CF93DF93A7
:100C8000FC01218120FF03C01185155F01C01BE01D
:100C9000082FC82FD92F8C2F801B811720F4899102
:100CA0000E94F403F8CFDF91CF911F910F91089527
:100CB0008EE792E00C943C068EE792E00E94470596
:100CC0006AEF8BEC92E00E94FC050C9487048EE2A4
:100CD00092E00E943C060C9487040E94520562E355
:100CE00089E792E00C94FC05CF92DF92EF92FF929D
:100CF0000F931F93CF93DF93EC018B017A0169016E
:100D00008091CF028823B1F18091D10281FF06C08A
:100D10008091CD0281608093CD022CC09091020120
:100D2000943041F1911124C0817091E08927209184
:100D30002F02217092278917D9F085E092E0FC01FB
:100D4000A4913196E491B0E0A053BD4FF0E0E25D94
:100D5000FD4F3C91208132130BC00296F2E08131AD
:100D60009F0769F780917D02816080937D0202C0B8
:100D70001092CF028091CE028430E1F08091020186
:100D80008430C1F00E94DC038823A1F0F701808148
:100D90009181892B61F00E94C703F7012081318185
:100DA000281B390B121613062CF011821082888131
:100DB00084608883F80180819181892B61F00E9491
:100DC000C703F80120813181281B390B1216130645
:100DD0002CF011821082888180628883F2E0CD3C01
:100DE000DF07A1F48091CE02843009F50E942D0422
:100DF00081111DC00E9438049091CD02882311F00A
:100E0000906101C098609093CD0211C08091020161
:100E1000843069F40E942D04811109C00E943804B5
:100E20009881882311F0906101C098609883F60141
:100E30008281882331F081E09381992319F080E049
:100E400001C081E080FF03C0888180688883F6014B
:100E500080818A3A19F0888180648883DF91CF91FC
:100E60001F910F91FF90EF90DF90CF9008952EE7A4
:100E700032E049EC52E06BEC72E08DEC92E00E94C3
:100E8000740641E152E06DEC72E08EEC92E00E945B
:100E90006A051092CD0208952EE232E049E752E051
:100EA0006BE772E08DE792E00E94740645EB50E03C
:100EB0006DE772E082E091E00E946A0510927D0287
:100EC0000895DF92EF92FF920F931F93CF93DF93DA
:100ED000FB011082FC012081222309F48CC0FF2435
:100EE000F3942181213009F4F12CF2E06E327F0776
:100EF00009F4F094EB018C01FC01328123816E52E4
:100F0000724091F0DC80D31276C0ED80E21273C0A3
:100F10008A8191E0882319F02B81211190E090FFC4
:100F200064C0E12CD12C61C0809103019091040137
:100F30004AEA48834F2D4370406C49833A832B83A0
:100F40008C839D83F80186818E8385818F83848144
:100F500088878085813410F4898701C01986DE0175
:100F6000CE010A96EFEF2D91E227F0E0EB5FFE4F06
:100F7000E491A817B907B9F7F0FE19C080E0998588
:100F8000891798F4282F30E0D801A20FB31F1996C3
:100F90009C91DE01A20FB31F1A969C93E927F0E003
:100FA000EB5FFE4FE4918F5FEACF865F01C08AE07E
:100FB000DE01A80FB11DEC938A81882331F081E016
:100FC0009B81992319F080E001C081E080FF13C06C
:100FD0008981833C29F49E81907F81E0903E09F0D5
:100FE00080E080FD08C0188206C06B810E940E055B
:100FF0003D2D2E2D9DCFDF91CF911F910F91FF9011
:10100000EF90DF9008959093040180930301089579
:1010100080910301909104010895CF93DF93EC0137
:101020000E9431058091CE02813071F4BE018EE7BD
:1010300092E00E94B8058091CD0282608093CD023B
:101040000E94370781E001C080E0DF91CF910895D1
:101050002091CE02223069F46EE772E00E946107AF
:101060008091CD0282608093CD020E94370781E09B
:10107000089580E0089520910201223069F46EE223
:1010800072E00E94610780917D02826080937D0200
:101090000E944C0781E0089580E00895CF93DF938C
:1010A000EC010E94310580910201813071F4BE0192
:1010B0008EE292E00E94B80580917D02826080936A
:1010C0007D020E944C0781E001C080E0DF91CF915A
:1010D000089581E090910201923009F080E0089536
:1010E0001092CE0282E0809302011092CF02E3E0E0
:1010F000F1E08FEF8083818308950F931F93CF9347
:10110000DF931F92CDB7DEB78091CF02811181C0EE
:101110000E946D04811102C010922D021AE00FEF9F
:10112000CE0101960E944A04882309F472C090916E
:101130002D02E981913059F018F0993081F01CC0EE
:10114000EA3A71F710932C0200932B0215C08E2FF0
:1011500086958695803381F010922D02E1CF8FEF36
:101160008E0F8034C8F78091D10280FF05C0809136
:101170002C028E0F80932C02A92FB0E0A053BD4FFC
:10118000EC9380912B02E827F0E0EB5FFE4FE491B7
:10119000E0932B0280912C02981337C010922D02FD
:1011A000E11137C08091D20290910301891711F0AB
:1011B00081112FC09091D30220910401921711F058
:1011C000911127C02091D402222319F12091D50238
:1011D0002223F9F0882329F081E0992319F080E097
:1011E00001C081E080FF0DC08091D102833C31F4C9
:1011F0009091D602907F81E0903E09F080E080FFE0
:1012000008C081E08093CF0204C09F5F90932D02BD
:1012100087CF0E9437070E944C070F90DF91CF9134
:101220001F910F9108958091CE028350823018F45F
:101230000E943707F8CF089580915703882369F0FB
:10124000909158039F5F9F3019F09093580302C00C
:101250001092580381508093570308958F929F9264
:10126000AF92BF92CF92DF92EF92FF920F931F93B4
:10127000CF93DF93CDB7DEB729970FB6F894DEBFD3
:101280000FBECDBF8C0120915903211104C0C801AC
:101290000E9431057EC0FC01C480D580E680F780C5
:1012A00060915A0370915B03FB0185919591A59123
:1012B000B491C816D906EA06FB0648F3215030E07F
:1012C000822F022E000C990B831B910937FD9395F9
:1012D00097FD019695958795830FFB0199E089020B
:1012E000E00DF11D112485909590A590B4908C147B
:1012F0009D04AE04BF0418F431E0380F07C0C814D1
:10130000D904EA04FB0438F42FEF280F231724F044
:101310008213D6CF01C0282FE9E02E02600D711D87
:10132000112449E050E0CE0101960E948C0CF80196
:1013300091818F81911103C0813039F4A8CF913010
:1013400009F0A5CF882309F4A2CF2D813E818981A0
:101350009A81AB81BC81820F931FA11DB11DF80141
:101360002085C20ED11CE11CF11C8C159D05AE051B
:10137000BF0508F48CCFE885F985309709F487CF4D
:10138000B801CE0101960995F8018081882309F4FE
:101390007ECF29960FB6F894DEBF0FBECDBFDF918A
:1013A000CF911F910F91FF90EF90DF90CF90BF9062
:1013B000AF909F908F900895CF92DF92EF92FF921F
:1013C0000F931F93CF93DF93CDB7DEB7C954D109E5
:1013D0000FB6F894DEBF0FBECDBF809157038823B0
:1013E00009F460C0E090580384E0E89E7001112485
:1013F000D701A55EBC4F6D018D919C91892BF1F1B8
:101400000E946908882309F44DC08E010F5F1F4FA9
:1014100089E4F80111928A95E9F7D601ED91FC91E2
:10142000C8010995C8010E943405882321F1F601FD
:1014300011821082DB800E940808D81218C0DC805C
:101440000E940808D91213C08981882319F0C801A5
:101450000E942E09F701E55EFC4FE280F3800E94B6
:101460001C09E114F104F1F0C801F7011AC0C80128
:101470000E943B0817C00E941C0914C0CE010196AF
:101480000E944E08882371F0D60112960D911C918E
:1014900013970E941C090115110521F0CE01019638
:1014A000F8010995C75BDF4F0FB6F894DEBF0FBE9A
:1014B000CDBFDF91CF911F910F91FF90EF90DF9003
:1014C000CF9008959C0190E02115310581F0F9013C
:1014D00089E0989FE00DF11D11244591559165918A
:1014E00074919F5F4C3F5F4F6F4F710581F7309351
:1014F0005B0320935A039093590308950C940308B7
:101500000E94080808950E94700810925B031092D0
:101510005A031092590310925803109257030895DA
:10152000CF93DF93CDB7DEB7C954D1090FB6F89486
:10153000DEBF0FBECDBF0E947D08CE0101960E9486
:101540000D08882359F08981882321F0CE01019666
:101550000E942E09CE0101960E9428080E94DC09F3
:10156000C75BDF4F0FB6F894DEBF0FBECDBFDF9174
:10157000CF9108950E946908811105C00E94DC097D
:101580000E947D08F7CF0C941309FC0160817181E2
:10159000828193810895DC01FB0194818C91981BD9
:1015A000892F9181992321F0913001F590E00EC0AF
:1015B000DB0119969085980F891739F0FA01E80F29
:1015C000F11D20812D938F5FF7CF0895392F380FAC
:1015D0002085921758F4DF01A90FB11D19962C919F
:1015E000DA01A30FB11D2C939F5FF0CF08950E94E5
:1015F00091040E948C0B0E94830A0E9497020E9411
:10160000CA04882349F00E94D1040E94E40B0E947E
:10161000900A0E94B402F3CF0E94B5020E94BA0A57
:101620000E94820C0C94F7040C94D5030E94DA03F8
:10163000109206011092050108950F931F93CF9306
:10164000DF931F92CDB7DEB70AE010E0F801E95A48
:10165000FD4FE491E98341E050E0B801CE010196ED
:101660000E94DA030F5F1F4F0834110579F71092BB
:101670000601109205010F90DF91CF911F910F91FC
:101680000895CF93DF9300D000D0CDB7DEB744E00C
:1016900050E0BE016F5F7F4F82E090E00E94D50373
:1016A0008B8180959981891308C06C8160959A819E
:1016B000691303C00E940E0502C09EE68FEF0F90D3
:1016C0000F900F900F90DF91CF9108950F931F937C
:1016D000CF93DF9300D000D0CDB7DEB78C010E944E
:1016E00010058983C8010E9413058A83998190950A
:1016F0009B8380958C8344E050E062E070E0CE01F3
:1017000001960E94DA030F900F900F900F90DF91D7
:10171000CF911F910F910895EF92FF920F931F9316
:10172000CF93DF9300D0CDB7DEB72AE0E22EF12CC5
:101730000FEF1FEF41E050E0BE016F5F7F4FC70129
:101740000E94D5038981082788E0A801569547950E
:1017500098012170332700FF02C028E034E88A0195
:1017600002271327815089F72FEFE21AF20A88E443
:10177000E816F104F9F60F3F2FEF120711F400E01D
:1017800010E042E050E0BE016F5F7F4FC7010E9452
:10179000D50389819A8124E5E216F10439F022E02B
:1017A000E20EF11C8F3F2FEF920759F3801791073C
:1017B00011F00E941D0B0F900F90DF91CF911F91A0
:1017C0000F91FF90EF900895EF92FF921F93CF93A8
:1017D000DF9300D000D01F92CDB7DEB78091050116
:1017E000909106018F3F2FEF920709F480C041E0EE
:1017F00050E0BE016B5F7F4F0A960E94D503209197
:101800000501309106012115310531F48FEF9FEF6D
:1018100090935D0380935C034D8180915C03909174
:101820005D03842748E0FC01F695E795BC016170F3
:10183000772780FF02C068E074E8CF0186279727EA
:10184000415089F790935D0380935C032F5F3F4F76
:101850002E33310529F0309306012093050147C04E
:101860002FEF3FEF30930601209305018F3F2FEFBD
:10187000920719F09C838B8302C01C821B8210E0AC
:1018800098E4E92EF12C42E050E0BE016F5F7F4FFB
:10189000C7010E94D50389819A818F3F2FEF92075C
:1018A00031F422E0E20EF11C1F5F173061F72B814B
:1018B0003C8182179307D9F08FEF9FEF9A8389833A
:1018C00042E050E0B701CE0101960E94DA031F5FAB
:1018D000173008F010E0612F70E06C5D7F4F660FED
:1018E000771F42E050E0CE0103960E94DA030F908A
:1018F0000F900F900F900F90DF91CF911F91FF905D
:10190000EF9008958091050190910601019619F0DC
:101910000E94E40BF7CF0895FB01DC0102C00590A3
:101920000D9241505040D8F70895DC01CB01FC01E5
:10193000F999FECF06C0F2BDE1BDF89A319600B428
:101940000D9241505040B8F70895DC01A40FB51F27
:101950004150504048F0CB01840F951F2E910E94BA
:10196000B60C41505040D0F70895262FF999FECF7C
:1019700092BD81BDF89A019700B4021639F01FBAE2
:1019800020BD0FB6F894FA9AF99A0FBE0895F8940C
:02199000FFCF87
:08199200010302FFFFFFFF004B
:00000001FF
